:0300000002510F9B
:0C510F0078FFE4F6D8FD75817702515658
:101B1D0020000A3C2E2E2E3E004950436F6E6E65FE
:101B2D0063745245510A004950436F6E6E6563747C
:101B3D00000A49504E6F41434B210A003E432C563B
:101B4D002C43432CC0E4E0EFF2E5F020D1E8EDEAC0
:101B5D00EEEC49500A003E432C4D41432C253032CA
:101B6D0062583A25303262583A25303262583A2559
:101B7D00303262583A25303262583A253032625846
:101B8D002C4D414320E0E4F0E5F10A003E432C5694
:101B9D0045522C20332E3220EEF220257320257352
:101BAD002CC2E5F0F1E8FF20495020ECEEE4F3EB18
:101BBD00FF0A004E6F762030312032303136003141
:101BCD00333A33363A3036003E432C4C442C505287
:101BDD004F473A2020202020202020202020202088
:101BED0020202020202020202020202020202020E8
:101BFD0020202020202020202020202020202020D8
:101C0D0020202020202020202020202020202020C7
:101C1D0020202020202020202CC4E0F2E020EFF016
:101C2D00EEF8E8E2EAE828F4E0E9EB290A003E2ABA
:101C3D002C312CCEF1EDEEE2EDFBE520EFE0F0E006
:101C4D00ECE5F2F0FB20F1E5F2E5E2EEE3EE20E863
:101C5D00EDF2E5F0F4E5E9F1E00A003E412C41300A
:101C6D00312C2562752E2562752E2562752E256205
:101C7D00752C495020E0E4F0E5F120E0E4E0EFF2CE
:101C8D00E5F0E00A003E412C4130342C2562752EE2
:101C9D002562752E2562752E2562752CCCE0F1EA34
:101CAD00E020F1E5F2E80A003E412C4130352C25CB
:101CBD0062752E2562752E2562752E2562752CD8BE
:101CCD00EBFEE70A003E2A2C312CCFE0F0E0ECE5EC
:101CDD00F2F0FB20EEE1ECE5EDE020EFEE20EFF091
:101CED00EEF2EEEAEEEBF3205544503937320A00AE
:101CFD003E412C4130322C2562752E2562752E25E4
:101D0D0062752E2562752C495020E0E4F0E5F12036
:101D1D00EEF1ED2E20F1E5F0E2E5F0E00A003E41B6
:101D2D002C4130332C2562752E2562752E2562755A
:101D3D002E2562752C495020E0E4F0E5F120F0E508
:101D4D00E72E20F1E5F0E2E5F0E00A003E422C53EB
:101D5D0030322C2562752CCEE1ECE5ED20F120F131
:101D6D00E5F0E2E5F0EEEC20E1E5E720EAE2E8F26D
:101D7D00E0EDF6E8E90A003E422C5330332C2562A3
:101D8D00752CCFE5F0E5E7E0EFF3F1EA20EFF0E8B1
:101D9D0020EFEEF2E5F0E520F1E2FFE7E820F1209B
:101DAD00F1E5F0E2E5F0EEEC0A003E422C5330385E
:101DBD002C2562752CCCE5E4EBE5EDEDFBE9204936
:101DCD005020EAE0EDE0EB28E7E0E4E5F0E6EAE0BC
:101DDD0020E4EE203520F1E5EA290A003E422C539D
:101DED0030352C2562752CCAE0EDE0EB20F8E8F0DB
:101DFD00EEEAEEE2E5F8E0F2E5EBFCEDEEE3EE20E7
:101E0D00EEE1ECE5EDE02028554450393733290A51
:101E1D00003E532C5330362C25303262582530324B
:101E2D006258253032625825303262582530326280
:101E3D005825303262582C4D414320E0E4F0E5F155
:101E4D0020F8E8F0EEEAEEE2E5F8E0F2E5EBFCED85
:101E5D00EEE3EE20EEE1ECE5EDE00A003E454E440A
:101E6D000A000A44756D7058202020202030302043
:101E7D003031203032203033203034203035203096
:101E8D003620303720303820303920304120304254
:101E9D00203043203044203045203046000A3A009F
:101EAD003A20000A000A44756D704420202020203D
:101EBD00303020303120303220303320303420305B
:101ECD003520303620303720303820303920304121
:101EDD002030422030432030442030452030460011
:101EED00457272206B657900526420656570726F62
:101EFD006D0A005264204D454D0A00526420436F17
:101F0D0064650A00577269746520436F64650A0041
:101F1D0044656275674950204F4E0A0044656275ED
:101F2D00674950204F46460A0044656275675573F0
:101F3D006572204F6E0A0044656275675573657250
:101F4D00204F46460A0044656275674D7367204F02
:101F5D006E0A0044656275674D7367204F46460AE9
:101F6D0000436F6E666967206C6F636B210A0057C3
:101F7D007220656570726F6D0A0020536176652061
:101F8D00656570726F6D210A00457272204D414377
:101F9D0021004C6F61643E3E002A00CEF8E8E1EA74
:101FAD00E00A00202D202575282575290A003C41C1
:101FBD0030313D003C4130323D003C4130333D003D
:101FCD003C4130343D003C4130353D003C21003C2E
:101FDD005330323D003C5330333D003C5330353DA2
:0D1FED00003C5330383D003C5330363D0081
:065BAA000174000172000D
:105B6200C28E438910758BFF758DB7D2ABD28E2250
:0A5B8100E4FEEEC39F50030E80F80F
:015B8B0022F7
:03001B0002507F11
:10507F00C0E0C083C082C0D0C28E758BFF758DB764
:10508F00201A0675A61E75A6E10572D216E5746084
:10509F000205740577E577540F7051E573D39401CA
:1050AF0040021573D222E577543F7012D2149070DC
:1050BF0008E0600A04F0E0D394B44002D21A907072
:1050CF0001E0600204F0906A7EE0600214F09070DC
:1050DF0009E0D394014003E014F03019020575E59F
:1050EF0076D394644004D21A80020576E571D39486
:1050FF000140021571D28ED0D0D082D083D0E03251
:100FAD00C291C290D2B5C21F7D027C007F07125B39
:100FBD002B8F27E527646060097D017F60125AC67B
:100FCD00D21FE4FDFC7F0B125B2B8F27E52730E64C
:100FDD00097D04E4FF125AEAD21F7D017C007F07D0
:100FED00125B2B8F27E5277008FD7FFF125AC6D2A3
:100FFD001F301F03126000C288C2A8C2AA758900E3
:10100D001254BB906CB9E0B4FA06A3E064CE607BD9
:10101D00E4F52774B12527F582E4346CF583E4F00B
:10102D000527E527B443EC906CB974FAF0A374CEA0
:10103D00F0A374CCF0906CBF740AF0E4A3F0A30499
:10104D00F0A3F0906CB574FFF0A3F0A3F0E4A3F05F
:10105D00906CD07403F0E4F527E5272401FFE43309
:10106D00FE74B12527F582E4346CF583E0FD125A48
:10107D00A20527E527C3944340DFE4F5A775A61E17
:10108D0075A6E1907FF0F0A3F080FE906CC4740320
:10109D00F0A374CCF0E4906CC3F0907006F0A3F064
:1010AD00124DADC2B5124A20C21A125800D21FC23B
:1010BD0021C220906EF17408F0906C2F7424F0E42E
:1010CD00A3F0906CB9E0906C31F0906CBAE0906C3C
:1010DD0032F0906CBBE0906C33F0906CBCE0906C97
:1010ED0034F0906CBDE0906C35F0906CBEE0906C7F
:1010FD0036F0757301E4906EF2F0C21BC21CC21D76
:10110D00C21E125A7B201F19AF277E007D03124B82
:10111D00F7E4FF124E7A7E1B7F1DE4FBFDFC1246A9
:10112D0033907008E060037401F0E4906A7EF0F58E
:10113D0075906EF0F0F576125B6275A70775A61EB9
:10114D0075A6E1D2AFC217E4F576906A7EE0700322
:10115D0012245C907009E06401701D908000741081
:10116D00F09080A874FFF0A3F0A3F0A3F0E49070CA
:10117D0009F0D21FC220C221908008E0F52730E48B
:10118D0005D21B7410F0E52730E508D21D908008BC
:10119D007420F0E52730E608D21C9080087440F0EA
:1011AD00E575C394034019908002E4F0908001F03E
:1011BD00908000F0E57594064006E4F57512580030
:1011CD009080A0E070031255B39080B8E0700312C8
:1011DD0055399080D0E070031257A4908000E070D4
:1011ED0013301B1012473A906CACEFF0D3940040C3
:1011FD0003120026908002E07006908000E06005EA
:10120D00D219021154C219E4F575906A7EE060039B
:10121D00021154201F12906EF3E0600C7E1B7F1F95
:10122D00124B0FE4906EF3F0301D12123FD2906C02
:10123D00ACEFF0D394004005E0FF125B72201C036D
:10124D000213E4123CD7906CACEFF0700302115412
:10125D00906CF0E054BF247F7003021336147003BA
:10126D0002130E2402600302137D201F077E1B7FD5
:10127D0026124B0F906FFCE060030213E4906CC8D4
:10128D00E07006906CCCE06067906FFDE0FF906CB5
:10129D00C8E0B50724906FFEE0FE906CC9E0B5067E
:1012AD0018906FFFE0FE906CCAE0B5060C907000D0
:1012BD00E0FE906CCBE06E6037906CCCE06F60031D
:1012CD000213E4906FFEE0FF906CCDE06F600302BF
:1012DD0013E4906FFFE0FF906CCEE06F600302139C
:1012ED00E4907000E0FF906CCFE06F60030213E4B8
:1012FD00C217906EF27401F0120021757301021382
:10130D00E4907008E060037401F0906FF5E0FF90D9
:10131D006CF2E06F60030213E4906FF5E004F0E40B
:10132D00F573906EF0F00213E43017030213E4909E
:10133D006CBFE07003021154906C2EE06008906C4D
:10134D00D0741EF08006906CD07403F0125BB1D295
:10135D0017E4F573906EF0F090700104F0E4906F67
:10136D00F4F0A3F0201F707E1B7F34124B0F8067AB
:10137D00907008E060037401F0301752906CF0E04B
:10138D0020E74B906CF2E0FF906FF4E0FE6F600D84
:10139D00906FFCE07007EE146F703C8013906FF44B
:1013AD00E004F0906CACE0FFD3940440031258EAD3
:1013BD0090697A7482F0A37401F0906CF2E09069F8
:1013CD007CF07E697F7A7D03125222021154201720
:1013DD0006906FFD74FFF0201703021507E573707B
:1013ED006E125994EF60237E6D7FF0906DF1E024C5
:1013FD0004FD125222906FFCE07009906CD0E0F564
:10140D0073021154E4F573021154907001E0D394FA
:10141D003C403C906FFCE07036906C2EE07030904C
:10142D00700104F0125B97E4906DF0F0A37412F06C
:10143D00906FF5E0906DF2F0A374FDF0906A7F630C
:10144D00A201906DF463A2017F121238518098129F
:10145D005B8C8F27E527B4011590697A7483F0E4CE
:10146D00A3F07E697F7A7D02125222021154E52784
:10147D00D39401401C90697A7483F0A37401F0E554
:10148D002724FEA3F07E697F7A7D0312522202117A
:10149D0054E57364016003021154906EF0E004F0A2
:1014AD00201F077E1B7F3E124B0F906EF0E0FFD387
:1014BD009401400B906CD0E0941E5003E004F0EFCB
:1014CD00C39405400DC217E4906EF2F01200210294
:1014DD0011547C6F7DFD906CC4E0FAA3E0FB7F029C
:1014ED001253B37E6D7FF0906DF1E02404FD125226
:1014FD0022906CD0E0F573021154E5736401600322
:10150D00021154906EF2E014606114700302160C17
:10151D0014700302161E24036003021154E4F575C2
:10152D00906FFCE0602D906CC8E0FCA3E0FDA3E0A3
:10153D00FEA3E0FF906FFD1230A9906CC47403F010
:10154D00A374CCF030B403021154906EF27401F018
:10155D000211549080027410F0906EF07401F075C9
:10156D007312906FFD74FFF0021154906FFDE060E7
:10157D005D906DF07480F0906DF27401F0E4A3F065
:10158D00A304F0A3743FF0A3747BF0E4F52774F784
:10159D002527F582E4346DF583747DF074F82527E5
:1015AD00F582E4346DF583E4F0E5272407906DF1C1
:1015BD00F07C6F7DFD906CC4E0FAA3E0FB7F02121E
:1015CD0053B37E6D7FF0E5272409FD125222906FF3
:1015DD00FCE06020E4906EF2F0125BB1D217E4F5FE
:1015ED0073906EF0F090700104F0E4906FF4F0A33E
:1015FD00F0021154E4906EF2F075731202115490D2
:10160D006EF27403F0F573C2B57FFF125B810211A8
:10161D0054E4906EF2F0125800757312021154805A
:01162D00FEBE
:01162E002299
:10002600906CF1E0B444047F0180027F00906CF094
:10003600E0B447047E0180027E00EE5F604A906C69
:10004600B9E0906CF2F0906CBAE0906CF3F0906CC2
:10005600BBE0906CF4F0906CBCE0906CF5F0906CAA
:10006600BDE0906CF6F0906CBEE0906CF7F0906C92
:10007600F17452F0906C2863A2019080A863A201EB
:100086007F061238510208F8906CACE0C394085011
:1000960003020901906CB9E0FF906CF2E06F600317
:1000A600020901906CBAE0FF906CF3E06F60030206
:1000B6000901906CBBE0FF906CF4E06F60030209ED
:1000C60001906CBCE0FF906CF5E06F6003020901E3
:1000D600906CBDE0FF906CF6E06F60030209019042
:1000E6006CBEE0FF906CF7E06F6003020901906C54
:1000F600F1E06444701A9080A8E0B4FF13906C2875
:1001060063A2019080A863A2017F06123851801075
:10011600906C2CE09080ACF0906C2DE09080ADF06F
:10012600907008E060037401F09070097464F090B8
:100136006CF17452F0906CF0E0646D600302029B07
:100146007BFF7A1B7949122C257BFF7A1B796390FA
:100156006CB9E0F530A3E0F531A3E0F532A3E0F5A4
:1001660033A3E0F534A3E0F535122C257530FF7581
:10017600311B7532C07533FF75341B7535CC7BFF6B
:100186007A1B7999122C257BFF7A1B79D5122C259F
:100196007BFF7A1C793B122C257BFF7A1C796890B1
:1001A6006CBFE0F530A3E0F531A3E0F532A3E0F54E
:1001B60033122C257BFF7A1C7992906CB5E0F530D2
:1001C600A3E0F531A3E0F532A3E0F533122C257B4D
:1001D600FF7A1C79B5906CB1E0F530A3E0F531A358
:1001E600E0F532A3E0F533122C257BFF7A1C79D299
:1001F600122C257BFF7A1C79FD906CC8E0F530A3A4
:10020600E0F531A3E0F532A3E0F533122C257BFFB0
:100216007A1D792B906CCCE0F530A3E0F531A3E0A4
:10022600F532A3E0F533122C257BFF7A1D79599020
:100236006FFCE0F530122C257BFF7A1D79849070D7
:1002460008E0F530122C257BFF7A1D79B7906C2ECD
:10025600E0F530122C257BFF7A1D79E9A215E433EF
:10026600F530122C257BFF7A1E791E906FF6E0F58D
:1002760030A3E0F531A3E0F532A3E0F533A3E0F5D2
:1002860034A3E0F535122C25123E5E7BFF7A1E79EB
:1002960069122C2522906CF0E0644C70737E1E7FF0
:1002A6006FFBFDFC124633906CF8E0F528A3E0F5F1
:1002B60029E4F52BE528906CFAF0A3E529F07E1EDB
:1002C6007FAA7C6C7DFA7B02124633E4F52A8529E7
:1002D60082852883E0FF74FA252AF582E4346CF5DA
:1002E60083EFF00529E52970020528052AE52AB4D9
:1002F60010DC7E1E7FAD7C6C7DFA7B1012463305CA
:100306002BE52BC3941040AC7E1E7FB0124B0F2200
:10031600906CF0E0646C7060F52C7E1E7FB2FBFD85
:10032600FC124633E4F52BE4906CFAF0A3E52CF0CE
:100336007E1E7FAA7C6C7DFA7B02124633E4F52A88
:10034600A82CE6FF74FA252AF582E4346CF583EFCF
:10035600F0052C052AE52AB410E67E1E7FAD7C6CDE
:100366007DFA7B10124633052BE52BC3940840B764
:100376007E1E7FB0124B0F22906CF0E0644B7061D2
:10038600F52A74E2252AF582E4346CF583E06032BE
:1003960074E2252AF582E4346CF583E0F460237474
:1003A600E2252AF582E4346CF583E0FF74F8252A09
:1003B600F582E4346CF583E0B50710052AE52AB426
:1003C60008C0906A7E7432F00208F8906CF07421CE
:1003D600F0301F030208F87E1E7FED124B0F020855
:1003E600F8906CF0E0B4521A201F077E1E7FF512BB
:1003F6004B0F906CF07472F07E6C7FF07D0812519A
:100406009B22906CF0E064497045201F077E1F7F99
:1004160000124B0F906CF8E0F528A3E0F529E4F5FF
:100426002A852982852883E0FF74FA252AF582E445
:10043600346CF583EFF00529E52970020528052AB5
:10044600E52AB480DC7E6C7FF07D8A12519B229077
:100456006CF0E064437046201F077E1F7F08124B36
:100466000F906CF8E0F528A3E0F529E4F52A852934
:1004760082852883E493FF74FA252AF582E4346C96
:10048600F583EFF00529E52970020528052AE52AF6
:10049600B480DB7E6C7FF07D8A12519B22906CF0DB
:1004A600E0645A7053201F077E1F7F11124B0F9076
:1004B6006CF8E0F528A3E0F5297C6C7DFA7B80AF2B
:1004C60029AE28125960E4F52A852982852883E415
:1004D60093FF74FA252AF582E4346CF583EFF00570
:1004E60029E52970020528052AE52AB480DB7E6CF9
:1004F6007FF07D8A12519B22906CF0E06444600389
:1005060002058F906CF8E0FF644470030208F8EF70
:10051600B4310CC21F7E1F7F1D124B0F0208F890CC
:100526006CF8E0B4300CD21F7E1F7F29124B0F02ED
:1005360008F8906CF8E0B4320CD2207E1F7F361299
:100546004B0F0208F8906CF8E0B4330CC2207E1F03
:100556007F44124B0F0208F8906CF8E0B4340CD2CA
:10056600217E1F7F53124B0F0208F8906CF8E0B4FF
:10057600350CC2217E1F7F60124B0F0208F8906C6B
:10058600F8E0FF12001E0208F8906A7EE070132061
:100596001F077E1F7F6E124B0F906CF07421F002C6
:1005A60008F8906A7E7432F0906CF0E0FFB4510463
:1005B600C2AF80FEEF64577045201F077E1F7F7C09
:1005C600124B0F906CF9E0906CACF0E4F52A906C4D
:1005D600ACE0FFE52AC39F40030208F874FA252A17
:1005E600F582E4346CF583E0FF906CF8E0252A246C
:1005F60027F582E4346BF583EFF0052A80D0906C02
:10060600F0E0645360030206B2201F077E1F7F8757
:10061600124B0F906CB9E0FF906B30E06F703C901E
:100626006CBAE0FF906B31E06F7030906CBBE0FF0E
:10063600906B32E0B50724906CBCE0FF906B33E022
:10064600B50718906CBDE0FF906B34E0B5070C90D1
:100656006CBEE0FF906B35E06F6016906CF0742115
:10066600F0301F030208F87E1F7F96124B0F020818
:10067600F8E4F52AE4F576AF2AFE7427252AF582F2
:10068600E4346BF583E0FD125AA2052AE52AC394E9
:10069600FE40E1C2AFE4907FF0F0A3F0907FFD74DE
:1006A600AAF0A374FFF0A37455F080FE906CF0E0FE
:1006B600644F705A906CF8E0F528A3E0F529E52917
:1006C6004528700A201F077E1F7F9F124B0F201F91
:1006D600077E1F7FA6124B0FE4F52A74FA252AF52A
:1006E60082E4346CF583E0852982852883F0052928
:1006F600E52970020528052AE52AB480DE907007F0
:10070600E02480F0907006E03400F00208F8906C67
:10071600F0E064457074906CF8E0FEA3E0FF907F13
:10072600F0EEF0A3EFF0D39400EE94044038907FFF
:10073600F0E0FEA3E0FF907006E0FCA3E0FD9FEC76
:100746009E4023E42FFFEE3401FED3ED9FEC9E5036
:1007560015C2AF907FFD74AAF0A374FFF0A3745581
:10076600F0E4F5A780FE7E1F7FA8124B0F7BFF7A71
:100776001F79B0907FF0E0F530A3E0F53190700678
:10078600E0F532A3E0F533122C25906CF0E06465B9
:100796006003020901906CF8E0FFA3E0907FF0CFC0
:1007A600F0A3EFF0E4F528F529D3907FF1E0952941
:1007B600907FF0E095284020E4F5762529FFE5288E
:1007C6003401FE852982852883E0FD125AA2052977
:1007D600E5297002052880D17E1F7FBB1252A9EF42
:1007E6004E6020120003906CBFEFF0120003906C75
:1007F600C0EFF0120003906CC1EFF0120003906C92
:10080600C2EFF07E1F7FC11252A9EF4E6020120088
:1008160003906CC8EFF0120003906CC9EFF0120061
:1008260003906CCAEFF0120003906CCBEFF07E1FC2
:100836007FC71252A9EF4E6020120003906CCCEFD6
:10084600F0120003906CCDEFF0120003906CCEEF27
:10085600F0120003906CCFEFF07E1F7FCD1252A9ED
:10086600EF4E6020120003906CB5EFF0120003907B
:100876006CB6EFF0120003906CB7EFF01200039025
:100886006CB8EFF07E1F7FD31252A9EF4E60201294
:100896000003906CB1EFF0120003906CB2EFF0120F
:1008A6000003906CB3EFF0120003906CB4EFF0E429
:1008B600F52AE4F576E52A2401FFE433FE74B12532
:1008C6002AF582E4346CF583E0FD125AA2052AE586
:1008D6002AC3944340DCC2AFE4907FF0F0A3F090CB
:1008E6007FFD74AAF0A374FFF0A37455F0E4F5A796
:0B08F60080FE7E6C7FF07D0812519B9D
:0109010022D3
:10592800AE07EEC39430400BEED394395005EE2405
:10593800D0FF22EEC39461400BEED394665005EE7F
:1059480024A9FF22EEC39441400BEED394465005A0
:08595800EE24C9FF22AF062274
:105B4800906C27E004F07006906C26E004F0906CEE
:0A5B580026E0FEA3E0FF125B0E2220
:10000300125B48125928EFC454F0FEC006125B4835
:08001300125928D0E02FFF2252
:10574700E4907262F0125B48907263EFF0C394309A
:105757004018E0FFD394395011907262E0247FF52E
:1057670082E4346AF583EFF08011907262E0247F5F
:10577700F582E4346AF583E4F0800C907262E00409
:10578700F0E0D3940840BE752B00752C00752D00F2
:0C579700E4F52E7B017A6A797F123B3327
:0157A30022E3
:0452A9008E2D8F2E89
:1052AD00906C26E4F0A374FFF0125B48EF606EF48F
:1052BD00606B852E82852D83E493B507EC752F01E8
:1052CD00E52E252FF582E4352DF583E493602590A9
:1052DD006C27E0252FFF906C26E03400FE125B0E4C
:1052ED00E52E252FF582E4352DF583E493B50704DE
:1052FD00052F80CCE52E252FF582E4352DF583E4A1
:10530D009370A6E52F24FFFFE434FFFE906C27E099
:10531D002FF0906C26E03EF07E007F0122E4FEFF30
:01532D00225D
:104DAD007E1F7FD91252A9EF4E70037F01227E1F05
:104DBD007FDC1252A9EF4E600C125B48EF24D090AD
:104DCD006FFCF08005E4906FFCF07E1F7FE21252C5
:104DDD00A9EF4E600C125B48EF24D0907008F08064
:104DED0005E4907008F07E1F7FE81252A9EF4E6027
:104DFD000C125B48EF24D024FF92158002C2157E61
:104E0D001F7FEE1252A9EF4E600C125B48EF24D0BB
:104E1D00906C2EF08005E4906C2EF0906CB963A22E
:104E2D0001906FF663A2017F0612385130153B7E5B
:104E3D001F7FF41252A9EF4E6030120003906FF6EF
:104E4D00EFF0120003906FF7EFF0120003906FF880
:104E5D00EFF0120003906FF9EFF0120003906FFA6C
:0D4E6D00EFF0120003906FFBEFF07F0022CA
:10585A00906EF1E0C3947C40027F0A906EF1E0FE04
:10586A0004F0742F2EF582E4346CF583EFF0BF0A4E
:10587A0027906EF1E0FF04F0742F2FF582E4346C68
:10588A00F583E4F0906EF1E0FF12532E906EF174FE
:09589A0008F0906C30E004F022EB
:105800009080007480F0906CB163A201F583F58202
:1058100063A2017F08123851906CB963A201908095
:105820008863A2017F0A1238519080927407F0A316
:1058300074D0F0A37406F0906CC3E0FF9080B1F0D8
:105840009080E1EFF09080957455F0A3F090800087
:0A5850007401F090800974F0F0225A
:1055B300908009E04410F09080A0E070609080A19A
:1055C3007482F09080A874FFF0A3F0A3F0A3F07F9F
:1055D300039080AEEFF0A374CBF09080007402F0E0
:1055E30090723C1230B50000000090723CE0908055
:1055F30040F090723DE0908041F090723EE09080E8
:1056030042F090723FE0908043F0A3E4F0A3F0A354
:0D561300F0A3F0908018F0A3F0A3F0A3F036
:015620002267
:1057A400908009E04440F09080D17482F07F0390AF
:1057B40080DEEFF0A374CCF09080027402F090725B
:1057C400401230B500000000907240E0908058F024
:1057D400907241E0908059F0907242E090805AF0CB
:1057E400907243E090805BF0A3E4F0A3F0A3F0A3F5
:0B57F400F0908030F0A3F0A3F0A3F0D1
:0157FF002287
:10553900908009E04420F09080B8E0706C9080B9C8
:105549007482F07F039080C6EFF07FCDA3EFF07FE8
:10555900039080C4EFF0A374CDF09080C074FFF085
:10556900A3F0A3F0A3F09080017402F090724412AA
:1055790030B500000000907244E090804CF09072C9
:1055890045E090804DF0907246E090804EF0907228
:1055990047E090804FF0A3E4F0A3F0A3F0A3F090CC
:0955A9008024F0A3F0A3F0A3F0AC
:0155B20022D6
:1053B3008C288D29A907EAFDE975F018A424ACFF10
:1053C300E5F034808F82F583EDF0EBFDE975F0189D
:1053D300A4FFAEF024ACFBEE34808B82F583A3ED07
:1053E300F08529828C83E0FDEF24A8FFEE3480FE54
:1053F3008F82F583EDF08529828C83A3E08F828EE3
:1054030083A3F0852982852883A3A3E0FDE975F0B2
:1054130018A424A8FFE5F03480FE8F82F583A3A3AC
:10542300EDF08529828C83A3A3A3E08F828E83A3CF
:04543300A3A3F0221D
:06519B008D2DAB07AA06F2
:1051A100908000E030E507906EF37401F022907278
:1051B1003CE0FCA3E0FDA3E0FEA3E0F5318E308DE1
:1051C1002F8C2EAE02AF038E838F8263A201E53056
:1051D100540744C0F58385318263A201AF2D123893
:1051E100C3E4FCFDFEE531252DF531EE3530F5301A
:1051F100ED352FF52FEC352EF52E908040E52EF074
:10520100A3E52FF0A3E530F0A3E531F09080007421
:1052110020F0AF31AE30AD2FAC2E90723C1230A9E0
:01522100226A
:065222008D28AB07AA066F
:10522800908002E030E507906EF37403F0229072EC
:1052380040E0FCA3E0FDA3E0FEA3E0F52C8E2B8D5F
:105248002A8C29AE02AF038E838F8263A201E52BDD
:10525800540744D0F583852C8263A201AF28123805
:10526800C3E4FCFDFEE52C2528F52CEE352BF52BAB
:10527800ED352AF52AEC3529F529908058E529F0ED
:10528800A3E52AF0A3E52BF0A3E52CF090800274A7
:1052980020F0AF2CAE2BAD2AAC299072401230A969
:0152A80022E3
:024E7A008F297E
:104E7C009080B8E07002FF22908001E06006741010
:104E8C00F07F0022907244E0FCA3E0FDA3E0FEA3BF
:104E9C00E0F52D8E2C8D2B8C2A906FF663A201E5FC
:104EAC002C540744C8F583852D8263A2017F06121A
:104EBC0038D9E52D2406F52DE4352CF52CE4352BCD
:104ECC00F52BE4352AF52A906EF463A201E52C54F7
:104EDC000744C8F583852D8263A201AF291238D906
:104EEC00E4FCFDFEE52D2529F52DEE352CF52CEDFC
:104EFC00352BF52BEC352AF52A90804CE52AF0A3BE
:104F0C00E52BF0A3E52CF0A3E52DF09080017420A7
:104F1C00F0AF2DAE2CAD2BAC2A9072441230A9AF51
:014F2C00295B
:014F2D002261
:10473A009081E0E0F52805280528052805280528A0
:10474A0005280528052805280528908010E0F52B5E
:10475A00A3E0F52CA3E0F52DA3E0F52E9081E1E08E
:10476A00F5280528052805280528052805280528E7
:10477A00052805280528908014E0F52FA3E0F530D8
:10478A00A3E0F531A3E0F532E531B52D08E532B500
:10479A002E037F0022E4F528E531540744E0F5832F
:1047AA0085328263A201906CF063A2017F081239FC
:1047BA0009906CF263A201906C2863A2017F061231
:1047CA003851906CF0E0F529A3E0F52AE4F5289039
:1047DA006CF0E0702AA3E024F8F528E53154074488
:1047EA00E0F58385328274082582F582E43583F503
:1047FA008363A201906CF063A201AF28123909AE5B
:10480A0029E4FCFDE532252AF532E5313EF531EDA4
:10481A003530F530EC352FF52F908014E52FF0A3C5
:10482A00E530F0A3E531F0A3E532F0908000744062
:03483A00F0AF28B4
:01483D002258
:103CD7009081E6E0F5280528052805280528052808
:103CE70005280528052805280528908028E0F52BB4
:103CF700A3E0F52CA3E0F52DA3E0F52E9081E7E0F6
:103D0700F528052805280528052805280528052854
:103D170005280528052890802CE0F52FA3E0F5302D
:103D2700A3E0F531A3E0F532E4F528E531B52D0A36
:103D3700E532B52E05C21C023E43E531540744F077
:103D4700F58385328263A201906CF063A2017F083C
:103D5700123909906CF0E0F529A3E0F52AE52A4528
:103D67002970099080027410F07F0022906FFDE0A7
:103D7700FFF46030906CF2E06F6003023E0A906FD0
:103D8700FEE0FF906CF3E06F7079906FFFE0FF90BB
:103D97006CF4E06F706D907000E0FF906CF5E06F71
:103DA7006031805F906CF2E0906FFDF0906CF3E013
:103DB700906FFEF0906CF4E0906FFFF0906CF5E080
:103DC700907000F0906CF6E0FFA3E0906CC4CFF029
:103DD700A3EFF0906CF0E0702AA3E024F8F528E553
:103DE70031540744F0F58385328274082582F582C1
:103DF700E43583F58363A201906CF063A201AF28D9
:103E0700123909AE29E4FCFDE532252AF532E53100
:103E17003EF531ED3530F530EC352FF52FAF2EAEC1
:103E27002DAD2CAC2BAB32AA31A930A82FD3123031
:103E37007840099080027410F07F002290802CE572
:103E47002FF0A3E530F0A3E531F0A3E532F0908041
:063E5700027440F0AF28E8
:013E5D002242
:103FD2009081E3E0F528052805280528052805280D
:103FE2000528052805280528052890801CE0F52BC2
:103FF200A3E0F52CA3E0F52DA3E0F52E9081E4E0FB
:10400200F528052805280528052805280528052856
:10401200052805280528908020E0F52FA3E0F5303B
:10402200A3E0F531A3E0F532E4F528E531B52D0A38
:10403200E532B52E05C21D024128E531540744E898
:10404200F58385328263A20190697E63A2017F0EAD
:1040520012391F90697EE0F529A3E0F52A9069865E
:10406200E0FFF4604A906FF6E0FEEF6E7079A3E035
:10407200FF906987E06F706F906FF8E0FF9069883A
:10408200E06F7063906FF9E0FF906989E06F70579D
:10409200906FFAE0FF90698AE06F704B906FFBE0DF
:1040A200FF90698BE06F703FE490698DF08008901B
:1040B200698D74FFF0D2D990697EE0702AA3E02462
:1040C200F2F528E531540744E8F583853282740E0F
:1040D2002582F582E43583F58363A20190697E63CC
:1040E200A201AF2812391FAE29E4FCFDE532252AD0
:1040F200F532E5313EF531ED3530F530EC352FF561
:104102002FAF2EAE2DAD2CAC2BAB32AA31A930A8DD
:104112002FD31230785006E52A4529700990800184
:104122007410F07F0022908020E52FF0A3E530F09C
:10413200A3E531F0A3E532F09080017440F0AF289E
:01414200225A
:044B0F008E318F3222
:104B1300908000E030E507906EF37401F02290720C
:104B23003CE0FCA3E0FDA3E0FEA3E0F5388E378D67
:104B3300368C35E538FFE5375407FEE42FF534EEC0
:104B430034C0F533853482F5837423F00534E534BA
:104B5300700205335333C7F582853383740AF00536
:104B630034E534700205335333C7906CB963A20143
:104B730085338385348263A2017F061238C37406AA
:104B83002534F534E43533F5338531838532826357
:104B9300A20185338385348263A2011238A7E4FC22
:104BA300FDFE90723CE0F8A3E0F9A3E0FAA3E02F46
:104BB300FFEE3AFEED39FDEC38FCEF2408FFE43E4E
:104BC300FEE43DFDE43CFC90723C1230A990723C43
:104BD300E0908040F090723DE0908041F090723E12
:104BE300E0908042F090723FE0908043F09080002C
:034BF3007420F03B
:014BF600229C
:0A4633008E2E8F2F8C308D318B32CC
:10463D00908000E030E507906EF37401F0229072E7
:10464D003CE0FCA3E0FDA3E0FEA3E0F5388E378D42
:10465D00368C35E538FFE5375407FEE42FF534EE9B
:10466D0034C0F533853482F5837423F00534E53495
:10467D00700205335333C7F582853383740AF00511
:10468D0034E534700205335333C7906CB963A2011E
:10469D0085338385348263A2017F061238C3740685
:1046AD002534F534E43533F533852E83852F826338
:1046BD00A20185338385348263A2011238A78F3915
:1046CD00EF2534F534E43533F533E53260178530B5
:1046DD008385318263A20185338385348263A20190
:1046ED00AF321238C3E53924082532F532FFE4FC28
:1046FD00FDFEE5382FF538EE3537F537ED3536F566
:10470D0036EC3535F535908040E535F0A3E536F0DE
:10471D00A3E537F0A3E538F09080007420F0AF38B2
:0C472D00AE37AD36AC3590723C1230A9AE
:01473900225D
:02532E008F41AD
:10533000908000E030E507906EF37401F0229072E7
:105340003CE0FCA3E0FDA3E0FEA3E0F5458E448D28
:10535000438C42E545FFE5445407FEE42FFFEE345D
:10536000C0906C2F63A201F5838F8263A201AF41CD
:105370001238C3E4FCFDFEE5452541F545EE354414
:10538000F544ED3543F543EC3542F542908040E578
:1053900042F0A3E543F0A3E544F0A3E545F0908097
:1053A000007420F0AF45AE44AD43AC4290723C1265
:0253B00030A922
:0153B20022D8
:064BF7008E308F31AB058A
:104BFD00908000E030E507906EF37401F022907222
:104C0D003CE0FCA3E0FDA3E0FEA3E0F5378E368D7E
:104C1D00358C34E537FFE5365407FEE42FF533EEDA
:104C2D0034C0F532853382F5837423F00533E533D3
:104C3D00700205325332C7F582853283EBF00533AE
:104C4D00E53370020532906CB963A201853283851C
:104C5D00338263A2017F061238C374062533F53300
:104C6D00E43532F5325332C7E530853382853283F0
:104C7D00F00533E533700205325332C7F5828532C4
:104C8D0083E531F00533E533700205325332C7E564
:104C9D0037240AF537E43536F536E43535F535E4A0
:104CAD003534F534908040E534F0A3E535F0A3E5D7
:104CBD0036F0A3E537F09080007420F0AF37AE36B4
:0A4CCD00AD35AC3490723C1230A9F2
:014CD70022BA
:10562100908009E04480F09080E97441F07F099016
:1056310080F6EFF0A37464F09080037402F0908020
:1056410003E020E1F99071381230B50000000090BC
:105651007138E0908064F0907139E0908065F0904D
:10566100713AE0908066F090713BE0908067F0A322
:10567100E4F0A3F0A3F0A3F090803CF0A3F0A3F03A
:02568100A3F094
:015683002204
:10483E009081E9E0F52E052E052E052E052E052E6E
:10484E00052E052E052E052E052E908034E0F52F13
:10485E00A3E0F530A3E0F531A3E0F5329081EAE074
:10486E00F52E052E052E052E052E052E052E052EB2
:10487E00052E052E052E908038E0F533A3E0F53495
:10488E00A3E0F535A3E0F536E535B53108E536B5E7
:10489E0032037F0022E4F52EE535540744F8F58304
:1048AE0085368263A20190713C63A2017F061239A4
:1048BE003790713CE064686014908038E52FF0A367
:1048CE00E530F0A3E531F0A3E532F0804C90713D78
:1048DE00E02402F52EE535540744F8F5838536823B
:1048EE0063A20190713C63A201AF2E123937E4FC32
:1048FE00FDFEE536252EF536EE3535F535ED35343E
:10490E00F534EC3533F533908038E533F0A3E534E8
:10491E00F0A3E535F0A3E536F09080037440F0AFD8
:01492E002E5A
:01492F002265
:024930008F2EC8
:104932009080E8E0640660037FFF22907138E0FC1B
:10494200A3E0FDA3E0FEA3E0F5328E318D308C2F83
:10495200E4FFFEFDFCAB32AA31A930A82FC312300E
:104962007870609081F9E0F52F907138E0FCA3E057
:10497200FDA3E0FEA3E0FFE4FAF9F8EF2401FFEA69
:104982003EFEE93DFDE83CFC9071381230A9907181
:1049920038E0FCA3E0FDA3E0FEA3E0FFE4F8EF248F
:1049A20001FFEA3EFEE93DFDE83CFC907138123021
:1049B200A9908064E0F52FA3E0F530A3E0F531A3E0
:1049C200E0F53290713C63A201E531540744D8F519
:1049D2008385328263A201AF2E1238F1E4FCFDFE20
:1049E200E532252EF532EE3531F531ED3530F53043
:1049F200EC352FF52F908064E52FF0A3E530F0A37E
:104A0200E531F0A3E532F09080037420F0AF32AECE
:0D4A120031AD30AC2F9071381230A97F000B
:014A1F002274
:105B0E00A2AF9223C2AF438E2075D2028F828E83B4
:0C5B1E00E0FFE4F5D2538EDFA22392AF2B
:015B2A002258
:105AA200E5D220E0FBA2AF9223C2AF43D2028F82A3
:105AB2008E83EDF075D25063D250A22392AFE5D21D
:035AC20020E0FBE6
:015AC50022BE
:1054BB00E4FDED2401FFE433FE125B0E74B12DF518
:1054CB0082E4346CF583EFF00DBD3FE6E4FDED2493
:1054DB007FFFE433FE125B0E74A72DF582E4346A72
:1054EB00F583EFF074A72DF582E4346AF583E07051
:1054FB001B74A72DF582E4346AF5837420F074A82D
:10550B002DF582E4346AF583E4F080040DBD80BE92
:10551B00E4906B26F0FDEDFF7E00125B0E74272DE1
:0D552B00F582E4346BF583EFF00DBDFEE971
:015538002250
:025960008B2D8D
:10596200A2AF9223C2AF85A22E53A2FE8E838F8254
:1059720005A28C838D82740912394DE52D53A2FE46
:1059820043A22012394F53A2DF852EA2A22392AF47
:01599200FF15
:0159930022F1
:105B2B00A2AF9223C2AF8C838D82EF12394D43A269
:0C5B3B002012394F53A2DFA22392AFFFCB
:015B4700223B
:025AC6008F2827
:105AC800A2AF9223C2AFE4F5838D82740612394DDA
:105AD800E52843A22012394F53A2DFA22392AF7FB9
:015AE80001BC
:015AE900229A
:025AEA008F2803
:105AEC00A2AF9223C2AFE4F5838D82740A12394DB2
:105AFC00E52843A22012394F53A2DFA22392AF7F95
:015B0C000197
:015B0D002275
:10377600A907E7FFA805EF93C3966008403B74FCD2
:103786002FFF80F00F08EF93C3966008402B74FB61
:103796002FFF80E00F08EF93C3966008401B74FA72
:1037A6002FFF80D00F08EF93D3966008400B74F973
:1037B6002FFF80C01F1F1F1F1FEF54FEF80303F7C4
:1037C600E893FC08E893FD08E893FE08E893FF22D7
:1037D60009E993C39D6008402974FB29F980F10922
:1037E600E993C39E6008401A74FA29F980E209E950
:1037F60093D39F6008400B74F929F980D3191919DE
:103806001919E9C313C313FF22740093F8ECC39884
:103816004024701F740193F8EDC398401970147416
:0E3826000293F8EEC398400E7009740393F8F5
:10383400EFC39840037F00227F0122EDF8E6F008F1
:10384400A3DFFA22EDF8E0F608A3DFFA22E0A3638F
:10385400A201F0A363A201DFF475A2002263A20116
:10386400F0A363A20122E0A363A201F0A363A20177
:10387400E0A363A201F0A363A201E463A201F0A3A5
:1038840063A201DFE175A20022E0A363A2016DFE41
:10389400936CFDEE058393FC158363A201DFEA7547
:1038A400A200227F00E493A363A201F00F600CA3A3
:1038B400E583C2E3F58363A20180EA75A20022E0F6
:1038C400A363A201F0A3E583C2E3F58363A201DF4E
:1038D400EE75A20022E0A363A201F0A3E583C2E493
:1038E400D2E3F58363A201DFEC75A20022E0A363B7
:1038F400A201F0A3E58344F8C2E5F58363A201DFE6
:10390400EC75A20022E583C2E3F583E0A363A20180
:10391400F0A363A201DFEE75A20022E583C2E4D224
:0A392400E3F583E0A363A201F0A322
:10392E0063A201DFEC75A20022E58344F8F583E083
:10393E00A363A201F0A363A201DFEE75A20022F938
:10394E0022C002C004C00612FFF0D006D004D0027E
:01395E002246
:104FDE004572724C656E210A000A496E49503A00BC
:104FEE00205544502054696D654750530A00200ADD
:104FFE00495054696D653A2000200A444154414796
:10500E0052414D3A20002049676E6F72650A2000AA
:10501E002043414E2054696D654750530A00205479
:10502E007261737353656E644552520A000ACEF86C
:10503E00C4EBE8EDFB43414E210A000A4572724172
:10504E00647243414E3A00205265496E69742043A2
:10505E00414E0A002043414E283029203E20544F15
:10506E00210A0020545520300A0020545520310AC0
:01507E000031
:03001E00E4FF22DA
:105A5300C2A9438902758C48758A4875D90475DBD8
:105A63004875DC4875DD4875DE48E4F5E9F5F9D29B
:085A7300D9C2DAD28CD2DE2286
:1059FA00C2D990701EE07013E5E92419F5EB30D78F
:105A0A0006E5F904F5FB2285F9FB22E5E924C8F548
:0E5A1A00EB30D706E5F904F5FB2285F9FB22F7
:1058A300C2D990701EE0702C303016E5E92432F531
:1058B300EB30D707E5F904F5FB800385F9FBC2302C
:1058C30022E5E92405F5EB30D706E5F904F5FB22DB
:1058D30085F9FB22E5E92432F5EB30D706E5F90437
:0758E300F5FB2285F9FB2211
:105A7B00125A5390701EE0C394645006125437129E
:105A8B0059FA120022D22FE4F557907136F0F546F1
:075A9B00F55BC230F5592252
:1058EA00EF24FCF546D3940D4010201F077E4F7F0E
:1058FA00DE124B0FE4F546D22D22906CF463A2011E
:10590A0090712663A201AF46123851C22D201F0D95
:0E591A007E4F7FE77C6C7DF4AB461246332255
:0F5B7200D3EF6480948D5006E55B70028F5B2249
:10245C0020D903022598202F03022598E55B7003F1
:10246C0002250B90697E540FFF7D48123848E548D1
:10247C006401706FE54B6401706990698DE0B4FF85
:10248C000ED231201F127E4F7FEE124B0F8009307F
:10249C003106E4F55B0225981259FA125684854DE3
:1024AC0011854E10854F0F85500E12429EE552F548
:1024BC0062E551F563AF097E007C037DE8122F1FA6
:1024CC00EF2563F563EE3562F562850C6B201F0D0D
:1024DC007E4F7FFC7C697D7EAB5B124633E4F55B03
:1024EC000225981259FA125684201F0D7E507F0730
:1024FC007C697D7EAB5B124633E4F55B022598E587
:10250C0046605590712AE02405F528D3940D4007B8
:10251C00E4F546D22D8075907126E528540FFF7D89
:10252C0048123848E54830E702D230E5486401707B
:10253C001A303117E54BB40112201F127E507F1454
:10254C007C697D7EAB5B1246338003125684125934
:10255C00FAE4F546D22D8034E558601E90700A548A
:10256C000FFF7D48123848E548B4010320310312AF
:10257C0056841259FAE4F558801220010C90701E02
:10258C00E0C394645003124CD81259FA1241438F91
:10259C0028EF70030226F7E4F559E54830E70AE521
:1025AC004BB41905D2D90226F71258A3E548640199
:1025BC007041E54B6401703BD231201F077E507F88
:1025CC001E124B0F854D11854E10854F0F85500EE9
:1025DC0012429EE552F562E551F563AF097E007C2F
:1025EC00037DE8122F1FEF2563F563EE3562F5626C
:1025FC00850C6BE55AC394C8501B301718741F25F3
:10260C005AF582E43470F583E528255AF55A7D484D
:10261C00AF2812383F301521E54820E71C906EF4A6
:10262C007D48AF2812383FAF28124E7AEF700A203F
:10263C001F077E507F2C124B0FE54854816003021C
:10264C0026F7E528D3940D4010301F030226F77EA1
:10265C00507F3B124B0F0226F7E54AD39407401FDD
:10266C00301F030226F7906A7F7D48AF2812383F4F
:10267C007E507F497C6A7D7FAB28124633806CE5A7
:10268C001230E662907261E0FF90571593FE547F12
:10269C0065487052EFA393654A704B907261E0C32A
:1026AC0013FF2448F582E43472F583E0703853123A
:1026BC003F907261E0FD744F2512F582E43462F5AF
:1026CC0083EEF0ED90571693FE74502512F582E4CC
:1026DC003462F583EEF074482FF582E43472F5839E
:1026EC007401F0431240AF2812284F302226906616
:1026FC00DDE0C394FA5003E004F030141590701E22
:10270C00E0C39464500C0559E55994F04004C2AFF1
:10271C0080FEC222201603022849740A2563F56341
:10272C00E43562F562FEAF63E4FCFD7B607AEAF9A6
:10273C00F8D31230625011E4F562F563056BE56B6A
:10274C00C3943C4003E4F56BE5576031D3940140EE
:10275C000415578028907136E004F0E0D3940340C0
:10276C000D201F077E507F55124B0F125A7B201FD6
:10277C00077E507F62124B0FE4F557D22FE558605D
:10278C0003022847302E3F90700A04F0A37408F01F
:10279C00A37480F0A37401F0A37406F0907121E08F
:1027AC0090700FF0907122E0907010F0907123E017
:1027BC00907011F0907124E0907012F0E4A3F0A3EB
:1027CC00F075580BC22E302C7290711FE07035E5ED
:1027DC0058703190700A7442F0A37408F090712014
:1027EC00E090700CF0907125E090700DF0A37401E6
:1027FC00F0755806201F077E507F71124B0F907199
:10280C001FE004F090711FE06402702FE558702BEC
:10281C0090700A7402F0A37408F0907120E090702C
:10282C000CF0A3F0A37401F0755806201F077E501E
:10283C007F78124B0F90711FE004F0C216121FFA32
:02284C00C214B4
:01284E002267
:10599400E55A602CE4906DF0F0A3E55AF0906FF5B1
:1059A400E0906DF2F0A37419F090701F63A201905F
:1059B4006DF463A201AF5A123851E4F55A7F012203
:0359C4007F00223F
:0B5B8C00302D05C22D7F01227F00227A
:0100210022BC
:065BB100E4F55AF546225E
:0A5B9700E4906A7FF0A3F0A3F0226F
:1056E6002043616E457247495400200A0045727294
:1056F6004C656E43616E21000A002043616E45725F
:1057060072434821000A205265714572722100C415
:1057160000C401C402C403C404C405C406C407C843
:1057260000C801C802C803C804C805C806C807C21D
:1057360000C201C202C203C204C205C206C20700F9
:015746000062
:10414300E59B541F6020201F1A7E567FE6124B0FFB
:10415300E59B541FFF7E007D03124BF77E567FF0D5
:10416300124B0FE4F59BE5BA30E010E4F5B375B1FB
:1041730080F5B2D22FF557907136F0E5CFF4700386
:1041830002429B752A01E4F529E5CFF4552A700311
:10419300024289E529C454F0F5B1E5B2547F6420A5
:1041A300600302425AE5B3540FF54C85BC48E5BDA4
:1041B300541FFF131313541FFFE5BD54E044184F5E
:1041C300F549E5BDC43354E0FFE5BE131313541F93
:1041D3004FF54AE5BEC43354E0FFE5BF1313135450
:1041E3001F4FF54B85A34D85A34E85A34F85A35044
:1041F30085A35185A35285A35385A354E4F5B22027
:10420300010FE548547EB5480843BDF875B35080A7
:104213000375B3D0E54C700AE548547EB548037F77
:104223000022300108E54830E7037F0022E54CD344
:104233009408401D201F177E567FF3124B0FAF4C7F
:104243007E007D03124BF77E567FFE124B0F7F00DD
:1042530022E54C2405FF22E5B2549F6023201F2052
:104263007E577F00124B0FAFB27E007D03124BF7D8
:10427300AFB37E007D03124BF77E567FFE124B0FCA
:10428300E4F5B275B3D0E52A25E0F52A0529E52939
:0A429300C39408500302418C7F0021
:01429D0022FE
:1056840090701EE0C39464505675B180E4F5B3F590
:10569400B28548BCE54AC4135407FFE54954E04FBA
:1056A400F5BDE54A33333354F8FFE54BC4135407CF
:1056B4004FF5BEE54B33333354F8F5BF854DA38521
:1056C4004EA3854FA38550A38551A38552A385532B
:1056D400A38554A3E54C540F2450F5B375570AC25F
:0256E4002F2273
:104CD80075B190E5B220E613201F107E577F0B12A6
:104CE8004B0FAFB27E007D03124BF7E4F5B3F5B27C
:104CF800E51230E615E4F512907261E02402F0E066
:104D0800905715937004907261F0744F2512F582D4
:104D1800E43462F583E0702D907261E0FFC31324E0
:104D280048F582E43472F583E070054312808015FB
:104D3800E4F512907261E02402F0E0905715937048
:104D480004907261F0E51230E721907261E0FF9003
:104D5800571593F5BCE4F5BDEFA393FF33333354F4
:104D6800F8F5BE75BF784312408036744F2512F5AA
:104D780082E43462F583E0F5BC75BD807450251279
:104D8800F582E43462F583E0FF33333354F8F5BE3B
:104D980075BF7805120512E512C394324003E4F595
:054DA8001275B350225A
:095BA100EF6003C29622D29622A5
:1054370043AB01C2E8C2EAE4FFEFC454F0F5B1C3DD
:10544700EF64809488500575B3D08003E4F5B3E426
:10545700F5B2F5BCF5BDF5BEF5BFF5C4F5C5F5C6A6
:10546700F5C7F5A3F5A3F5A3F5A3F5A3F5A3F5A351
:10547700F5A30FBF0EC390701EE0FE25E0F5B475CF
:10548700B50C75B66C75A11275AB0275C13E75C3C7
:10549700FF75C203E4907261F0751280FF7F199067
:1054A7007248E4F0A3DFFCE4FF7F3290624FE4F040
:0354B700A3DFFC74
:0154BA0022CF
:10395F000000000000000000000000000000000058
:10396F003FF3630041D5E80043B71B8045984F00F4
:10397F0047798280495C07804B3D3B004D1E6E802E
:10398F004EFFA20050E2270052C35A8054A48E006B
:10399F005685C180586846805A497A005C2AAD80A6
:1039AF005E0BE1005FEE660061CF998063B0CD00E2
:1039BF0065920080677485806955B9006B36EC801D
:1039CF006D1820006EFAA50070DBD8800000000093
:1039DF000028DE80004DC8800076A700009E3400CE
:1039EF0000C7123000EE9F8001177E0001405C80FF
:1039FF000167E9800190C80001B8550001E13380EB
:103A0F00000000000028DE80004F1A000077F880C9
:103A1F00009F858000C8640000EFF1000118CF807F
:103A2F000141AE0001693B000192198001B9A680E6
:103A3F0001E2850000000000000151800002A30098
:103A4F000003F48000054600000697800007E90098
:103A5F0000093A80000A8C00000BDD80000D2F005A
:103A6F00000E8080000FD20000112380001275001D
:103A7F000013C68000151800001669800017BB00E0
:103A8F0000190C80001A5E00001BAF80001D0100A2
:103A9F00001E5280001FA4000020F5800022470066
:103AAF00002398800024EA0000263B8000278D0029
:103ABF000028DE800000000000000E1000001C2017
:103ACF0000002A30000038400000465000005460CB
:103ADF00000062700000708000007E9000008CA0DB
:103AEF0000009AB00000A8C00000B6D00000C4E0EB
:103AFF000000D2F00000E1000000EF100000FD20F8
:103B0F0000010B3000011940000127500001356002
:103B1F0000014370000151801F1C1F1E1F1E1F1F1D
:043B2F001E1F1E1F18
:1043F900E50825E025E0245FF582E43439F58312E8
:1044090030898F118E108D0F8C0EE508540370289A
:10441900E50D25E025E0240BF582E4343AF5831215
:104429003089EF2511F511EE3510F510ED350FF541
:104439000FEC350EF50E8026E50D25E025E024D795
:10444900F582E43439F583123089EF2511F511EE3F
:104459003510F510ED350FF50FEC350EF50EE50AB3
:1044690025E025E0243FF582E4343AF583123089CA
:10447900EF2511F511EE3510F510ED350FF50FECAF
:10448900350EF50EE50BC3940C402AE51124C0F551
:1044990011E51034A8F510E4350FF50FE4350EF5E4
:1044A9000EE50B24F4FF7E007C0E7D10122F1FAA4F
:1044B90006AB07800FAF0B7E007C0E7D10122F1FFD
:1044C900AA06AB07AE02E4FCFDE5112BF511E510D8
:1044D9003EF510ED350FF50FEC350EF50EE50C75C3
:1044E900F03CA4FFAEF0E4E5112FF511E5103EF51F
:1044F90010ED350FF50FEC350EF50EE4FEE511253F
:1045090009F511EE3510F510ED350FF50FEC350EF7
:02451900F50E9D
:01451B00227D
:10429E00907264E0F50825E025E0245FF582E434B1
:1042AE0039F583E508D3941F501DAF11AE10AD0F35
:1042BE00AC0E12380FEF700F74042582F582E435C0
:1042CE0083F583050880DC74FC2582F58274FF3546
:1042DE0083F583AF82123099C3E5119BF511E5107A
:1042EE009AF510E50F99F50FE50E98F50E1508E500
:1042FE000814907264F0E50854037005903A0F802C
:10430E00039039DB750D01AF11AE10AD0FAC0E126F
:10431E00380FEF701474042582F582E43583F5832B
:10432E00050DE50DD3940C40DE74FC2582F58274E8
:10433E00FF3583F583AF82123099C3E5119BF511DA
:10434E00E5109AF510E50F99F50FE50E98F50E1597
:10435E000D903A43AF11AE10AD0FAC0E7B007A004C
:10436E00797C1237D68F0AEF25E025E02443F582BB
:10437E00E4343AF583123099C3E5119BF511E5103B
:10438E009AF510E50F99F50FE50E98F50E050A90C2
:10439E003AC3AF11AE10AD0FAC0E7B007A00795C54
:1043AE001237D68F0BEF25E025E024C3F582E434D7
:1043BE003AF583123099C3E5119BF511E5109AF584
:1043CE0010E50F99F50FE50E98F50EAE10AF117CB6
:1043DE00007D3C122F318D09AE10AF117C007D3C5B
:0B43EE00122F318E108F1185110C2250
:10162F003E2A2C312CCFE0F0E0ECE5F2F0FB20F37A
:10163F00EFF0E0E2EBFFFEF9E5E3EE20EAEEEDF28C
:10164F00F0EEEBEBE5F0E020CACF20C8F1E5F2FCBD
:10165F000A003E4C2C6B30312C25732C43EAEEF0F4
:10166F00EEF1F2FC20EDE020F8E8EDE52043414EED
:10167F002C30202D20353030EAE1283530EC292C64
:10168F0031202D203530EAE128353030EC290A00A1
:10169F0030202D20353030EAE1283530EC2900316B
:1016AF00202D203530EAE128353030EC29003E423C
:1016BF002C6330312C2562752CC2F2EEF0E8F7ED79
:1016CF00FBE920EAEEEDF2F0EEEBEBE5F020EDE0DA
:1016DF0020F8E8EDE50A003E2A2C312CCFE0F0E0AF
:1016EF00ECE5F2F0FB20EFF0EEF2EEEAEEEBE020AD
:1016FF00CCDDCA203837302D352D313034283130FC
:10170F0031290A003E4C2C6B30352C256C752C285A
:10171F0031303129D1EAEEF0EEF1F2FC20EEE1ECBE
:10172F00E5EDE020EDE020EFEEF0F2F32C3130307C
:10173F002C3230302C3330302C3630302C3132309C
:10174F00302C323430302C343830302C3936303075
:10175F002C31393230302C33383430302C35373659
:10176F0030302C3131353230300A003E532C6B3053
:10177F00362C2562752C2831303129CDEEECE5F071
:10178F0020F1F2E0EDF6E8E80A003E532C6B30371B
:10179F002C2562752CC0E4F0E5F120415344550A25
:1017AF00003E532C6B30382C256C752CCDE0F7E0B8
:1017BF00EBFCEDFBE920E0E4F0E5F120D2D10A00EB
:1017CF003E532C6B30392C256C752CCDE0F7E0EBAC
:1017DF00FCEDFBE920E0E4F0E5F120D2C8D20A00ED
:1017EF003E532C6B31302C256C752CCDE0F7E0EB94
:1017FF00FCEDFBE920E0E4F0E5F120D2C8C80A00D7
:10180F003E532C6B31312C256C752CCDE0F7E0EB72
:10181F00FCEDFBE920E0E4F0E5F120D2D30A003E35
:10182F00532C6B31322C2562752CD0E0E7ECE5F0B0
:10183F0020C0D1C4D328312032290A003E532C6B4B
:10184F0031332C2562752CD0E0E7ECE5F020EFF07A
:10185F00E8F7E8EDFB20EFE5F0E5E4E0F7E8283105
:10186F002032290A003E532C6B31342C2562752C03
:10187F00D0E0E7ECE5F020E0E4F0E5F1E020EEE188
:10188F00FCE5EAF2E028322033290A003E422C6BB5
:10189F0031352C2562752CCFE5F0E5E4E0E2E0F27E
:1018AF00FC20F6E8EAEB20D2D12DD2C8D20A003EB6
:1018BF00422C6B31362C2562752CCFE5F0E5E4E038
:1018CF00F7E020D2C8D220F120E2F0E5ECE5EDE51B
:1018DF00EC0A003E422C6B31382C2562752CCFE57B
:1018EF00F0E5E4E0F7E020D2C8D220EAE0EA20EC0D
:1018FF00E0F1F8F22FEDEEF0EC0A003E532C6B31D5
:10190F00372C2562752C2831303429CAEEEB20EFA5
:10191F00E0EAE5F2EEE220EDE020EAE2E8F20A008A
:10192F003C21003C6B30313D003C6330313D003C8D
:10193F006B30353D003C6B30363D003C6B30373DF6
:10194F00003C6B30383D003C6B30393D003C6B3117
:10195F00303D003C6B31313D003C6B31323D003C42
:10196F006B31343D003C6B31333D003C6B31353DC9
:10197F00003C6B31363D003C6B31373D003C6B31E9
:10198F00383D000A414F75743A0043414E2054557B
:10199F00205265710A0043414E205455204F4B0A87
:1019AF0000496E69745443500A004C697374656E34
:1019BF005443500A00534F434B5F5443505F4553BA
:1019CF005441424C49534845440A004E6F204B56F0
:1019DF005421205443502041626F72740A002054E6
:1019EF00552054696D654F5554210A000A2D3E202C
:1019FF00000A4173496E000A3ED1E1F0EEF1CAE0F0
:101A0F00EDE0EBE0203A3C28CAE2F229000A3ED191
:101A1F00E1F0EEF1CFF0EEF6E5E4F3F0203A3C28FA
:101A2F00CAE2F229000A3E003A3C28CAE2F2290033
:101A3F000A3ED1F2E0F2F3F1CAE0EDE0EBE03F2035
:101A4F003A3C28CAE2F229000A3EC7E0EFF0EEF175
:101A5F003A003C28CDE5F2C4E0EDEDFBF529003E60
:101A6F003F3F3F3A0020D2D3200020C2FBE1EEF0EF
:101A7F00200020C8F1EFEEEBEDE8F2FC200020CEC5
:101A8F00F2ECE5EDE0200020C2F0E5ECFF200020B5
:101A9F00CEEFF0EEF1200020C7E0E2E5F0F8E5ED43
:101AAF00E8E5C8EDE8F6E8E0EBE8E7E0F6E8E8207F
:101ABF000020CAE2E8F2D2D3200020CEF8E8E1EA13
:101ACF00E0D2D3200020D2D320C3EEF2EEE2EE20FC
:101ADF000020D2D320C2FBEFEEEBEDE5EDEE2000C0
:101AEF0020D2D1F1200020C0EAF2E2F6CEEFF0EEE4
:101AFF00F1E0200020D2D1F6200020D2C8D2F6206B
:0E1B0F000020D2C8C8200020D2C8D2F1200089
:0300230002451C77
:0D451C00C0E0C0F0C083C082C0D075D018D0
:104529002098030245EDC298757401AF99300603CE
:10453900024628D291200228BF680DD202D20E75F8
:1045490064007568000245EDEF641060030245EDF3
:10455900D202D20F7570027568037564000246288D
:10456900E56870078F700568024628E568B4010F91
:10457900E570B51F050568024628C202024628E50E
:1045890068B4020AEF646860CEC202024628E56890
:10459900B4031E74382569F582E43467F583EFF0B6
:1045A90005692564F5641570E57070737568048094
:1045B9006EE568B4040DE564B51F0405688060C242
:1045C90002805CE568B4051CBF160ED206856970C9
:1045D900756900C202C2918046C20FC20E75690098
:1045E900C202803B30993830033390620DE0FFE519
:1045F9006CC39F400DC203D210E4FF125BA1C290AD
:10460900801BD2907478256CF582E43468F583E0D8
:0F461900F56F526FA2D0929B856F99056CC29975
:0B462800D0D0D082D083D0F0D0E032A0
:103E5E007BFF7A16792F122C2590701EE070147548
:103E6E0030FF75311675329F7BFF7A167961122CF1
:103E7E002580127530FF7531167532AE7BFF7A16BE
:103E8E007961122C257BFF7A1679BDA201E433F5F8
:103E9E0030122C257BFF7A1679E6122C2590697844
:103EAE00E0FEA3E0FFC3E49FFFE49EFEAB07FA3300
:103EBE0095E0F9F87F007E8C7D0A7C00122FC28F70
:103ECE00338E328D318C307BFF7A177913122C257D
:103EDE007BFF7A17797A9064D2E0F530122C257B2D
:103EEE00FF7A177999906100E0F530122C257BFF4F
:103EFE007A1779B09064D3E0FEA3E0FFE48F338E9F
:103F0E0032F531F530122C257BFF7A1779CF90627E
:103F1E000BE0FEA3E0FFE48F338E32F531F5301265
:103F2E002C257BFF7A1779EF906209E0FEA3E0FF64
:103F3E00E48F338E32F531F530122C257BFF7A1853
:103F4E00790F9066E8E0FEA3E0FFE48F338E32F542
:103F5E0031F530122C257BFF7A18792EA205E43329
:103F6E0004F530122C257BFF7A18794BA204E4332A
:103F7E0004F530122C257BFF7A187974A20BE433EA
:103F8E002402F530122C257BFF7A18799BA20AE4C5
:103F9E0033F530122C257BFF7A1879BEA212E4334A
:103FAE00F530122C257BFF7A1879E2A209E433F55D
:103FBE0030122C257BFF7A19790A906737E0F5309D
:043FCE00122C25226A
:10354C007E197F2F1252A9EF4E70037F0122E49057
:10355C00701EF07E197F321252A9EF4E6015125B6D
:10356C0048BF310690701E740AF0BF320690701E70
:10357C007464F07E197F381252A9EF4E600D125709
:10358C0047EC4D4E4F24FF92018002C2017E197F01
:10359C003E1252A9EF4E6023125747A804A905AA60
:1035AC0006AB077F007E8C7D0A7C00122FC2123086
:1035BC0054906978EEF0A3EFF0800A90697874FD6E
:1035CC00F0A374C0F07E197F441252A9EF4E600A2A
:1035DC001257479064D2EFF080069064D27401F0D9
:1035EC007E197F4A1252A9EF4E600A12574790611A
:1035FC0000EFF080089064D2E0906100F07E197FBB
:10360C00501252A9EF4E600D1257479064D3EEF052
:10361C00A3EFF080089064D3E4F0A304F07E197F4C
:10362C00561252A9EF4E600D12574790620BEEF0F6
:10363C00A3EFF0800A90620B7403F0A374E9F07EA0
:10364C00197F5C1252A9EF4E600D12574790620918
:10365C00EEF0A3EFF0800A906209740BF0A374B93A
:10366C00F07E197F621252A9EF4E600D12574790EF
:10367C0066E8EEF0A3EFF0800A9066E87407F0A31A
:10368C0074D1F07E197F681252A9EF4E601C12574C
:10369C0047EF24FFFFEE34FFFEED34FFFDEC34FF6B
:1036AC00FC4D4E4F24FF92058002C2057E197F6EA1
:1036BC001252A9EF4E601C125747EF24FEFFEE3456
:1036CC00FFFEED34FFFDEC34FFFC4D4E4F24FF921A
:1036DC000B8002C20B7E197F741252A9EF4E601C34
:1036EC00125747EF24FFFFEE34FFFEED34FFFDECE5
:1036FC0034FFFC4D4E4F24FF92048002C2047E190D
:10370C007F7A1252A9EF4E600D125747EC4D4E4F77
:10371C0024FF920A8002D20A7E197F801252A9EFEE
:10372C004E600D125747EC4D4E4F24FF9212800203
:10373C00D2127E197F861252A9EF4E600A12574799
:10374C00906737EFF080069067377401F07E197F31
:10375C008C1252A9EF4E600D125747EC4D4E4F2470
:09376C00FF92098002C2097F00EE
:013775002231
:104A2000E4F56C74DE256CF582E43466F583E4F01D
:104A300074D5256CF582E43466F583E4F074C925F9
:104A40006CF582E43463F583E4F0056CE56CB4083E
:104A5000D2E4F56C7438256CF582E43468F583E4AF
:104A6000F0056CE56CB440ECE4F56C7481256CF5F4
:104A700082E43462F583E4F0056CE56CB480ECE428
:104A8000907137F0C22CF56EF56D907264F0C20330
:104A9000C2089066E7F0C211C207C210C202C20685
:104AA000F56C90620DF0F560F569F574C200C21303
:104AB000C20D90697874FFF0A374F4F07565FF90EF
:104AC00061017402F0A3F090624EF012354CE4F5EF
:104AD00012C291C290C2ADF5C9D2CDD2CCC2C9C268
:104AE000CAF5CDF5CC906978E0F5CBA3E0F5CA85A1
:104AF000CBCD85CACCD29FD29ED29CD2CAC2ACC2E8
:0F4B000098C29975B81075B710D2AC1256212211
:024F2E008F2EC4
:104F3000E4FF7C617D03FEEEC3952E50120DEDAAB9
:104F40000470010C14F5828A83E02FFF0E80E80DB7
:104F5000EDAA0470010C14F5828A83EFF00DEDAE1A
:104F60000470010C14F5828E837416F0052E052E44
:104F70007E687F787C617D03E52EB4040E8F828E7F
:104F8000837410F00FBF00010E80328F828E837405
:104F900068F00FBF00010EE52E24FEFB8F828E838A
:104FA000F00FBF00010E8F828E83EBF00FBF000168
:104FB0000E8F828E837468F00FBF00010E8C838D7C
:104FC0008263A2018E838F8263A201AF2E123851B9
:0D4FD000E52EB4040304FF22E52E2404FFA7
:014FDD0022B1
:1059C70020032F124F2E90620DEFF030210D7E191C
:1059D7007F927C687D78E0FB1246337F01125BA1E2
:1059E700E5606003F57122E49066DDF0F56CD203A3
:0359F700D2992220
:02284F008F29CF
:10285100E54954E324DF7003022A1924DF700302DF
:1028610029BF1470030229EF24E37003022A911493
:102871007003022A91147003022B8A24E2605D2402
:10288100606003022BC2E54864446003022BC2E589
:102891004AD394074003022BC2E54C64066003024D
:1028A1002BC2300A1174D5254AF582E43466F583CA
:1028B100E04481F0800F74D5254AF582E43466F551
:1028C10083E04401F0E54A25E025E0240BF582E4AC
:1028D1003467F5837D4D7F0412383F22E548644417
:1028E1006003022BC2E54AD394074003022BC2E5E1
:1028F1004C64086003022BC2752901E54B5407FFA4
:10290100E529A807088002C333D8FCF529740825F6
:102911006EF56EB56D067408256DF56DE54B541FAA
:10292100FFE54AC43354E02FFE7400256EF582E4BE
:102931003460F583EEF0E54BC394805038EF131308
:1029410013541FFFE54A25E025E0240BF582E4340A
:1029510067F583E5822FF582E43583F583E0FFE5B2
:1029610029F4FEEF5EF07401256EF582E43460F522
:1029710083E4F08036E54B541FFF131313541FFFFC
:10298100E54A25E025E0240BF582E43467F583E58B
:10299100822FF582E43583F583E04529F074012522
:1029A1006EF582E43460F5837401F07402256EF5EE
:1029B10082E43460F5837D4D7F0612383F22202C5E
:1029C10003022BC2E54864426003022BC2E54B645B
:1029D100036003022BC290711FE0B401037405F080
:1029E100301F03022BC27E197F99124B0F22202C1C
:1029F10003022BC2E54864426003022BC2E54B642B
:102A0100016003022BC2201F077E197FA5124B0F05
:102A1100E54E04907137F022E54864446003022BCF
:102A2100C2E54AD394014003022BC2E54C6408601D
:102A310003022BC2E54A7007E54B14F52A8006E52F
:102A41004B241FF52AE52A75F004A424D2F58274DB
:102A51006335F0F5837D4D7F0412383FE52A75F02B
:102A610004A424C9F582746235F0F5837D517F0495
:102A710012383F74C1254AF582E43462F5837481CA
:102A8100F07481252AF582E43462F5837401F02221
:102A9100E54864486003022BC2E54AD3940740032A
:102AA100022BC2E54B547FFF941C4003022BC2E56D
:102AB1004C64086003022BC274C9254AF582E434D0
:102AC10063F583E0F50CEF1313543FF50AE54A75FE
:102AD100F008A4250AF50DE50C30E657540FB50AA8
:102AE1002D301216E50C54074490FF74C9254AF5A0
:102AF10082E43463F583EFF08014E50C540744104D
:102B0100FF74C9254AF582E43463F583EFF030128E
:102B1100117438250DF582E43468F583E054FEF034
:102B210080207438250DF582E43468F583E0440390
:102B3100F0800F7438250DF582E43468F583E044A4
:102B410003F075F040E54AA424D5F582E5F034643C
:102B5100F583E54B547F75F0021230E67D4DAF4CA5
:102B610012383F30315B740E250DF582E43462F585
:102B710083E56BF0E50D25E02486F582E43461F50B
:102B810083E562F0A3E563F022E54864487032E52D
:102B91004AD39407502BE54B540F144440FF74C99A
:102BA100254AF582E43463F583EFF0E54A25E02513
:102BB100E024EAF582E43466F5837D4D7F04123822
:012BC1003FD4
:012BC20022F0
:101FFA002014030220809080E8E0700F12562130EE
:10200A0021077E197FB0124B0FC20C9080E8E0B412
:10201A000E159080037408F03021077E197FB912DB
:10202A004B0FC20C7561559080E8E0B40614200C81
:10203A00113021077E197FC4124B0FE56A700375B0
:10204A006A0AE56A6013D56A109080037410F0304A
:10205A0021077E197FDA124B0FC214302C189062B6
:10206A0006E004F0E0D39414400C201F077E197F89
:10207A00ED124B0FC22C9066E7E0704B90670AE0B6
:10208A0004F0E0FFD394074007E56160037561033C
:10209A00EF540790670AF0E0FF24C9F582E434633D
:1020AA00F583E0FE30E72074C92FF582E43463F546
:1020BA0083EE547FF074C92FF582E43463F583E02C
:1020CA00540F049066E7F020112A906207E004F0AA
:1020DA00E0543FF0E0FF2438F582E43468F583E009
:1020EA00FE30E010D21174382FF582E43468F5839B
:1020FA00EE54FEF02007269066E6E004F0E0543F36
:10210A00F0E0FF2481F582E43462F583E0600ED2C8
:10211A000774812FF582E43462F583E4F020082AFB
:10212A00906208E004F0E05407F0E0FF24D5F5825D
:10213A00E43466F583E0FE30E71074D52FF582E4C7
:10214A003466F583EE547FF0D208300C63E56A708A
:10215A005F7E717F421209028F29E52960529071D0
:10216A003EE55FF0E55EA3F0A3E55DF0E55CA3F074
:10217A003005020529300B0205293004020529E53C
:10218A0029240490713DF0E5292406FF1249307490
:10219A0002255FF55FE4355EF55E9063D1E004F0F9
:1021AA00906737E0FF9063D1E0C39F4003756A08E8
:1021BA0012483E8F29E529700302228C30210C7EB9
:1021CA00197FFB7C717D3CFB12463390713EE0B473
:1021DA000722740BF07F06124930E4F55EF55FF5CD
:1021EA005CF55DD20CF56A9063D1F0907137F0C25C
:1021FA002C75615590713EE0B443087483F07F06F4
:10220A0012493090713EE0B4130A7423F07F06122B
:10221A004930C20C90713EE0FFB40107E4F56A90C0
:10222A0063D1F0EF20E05DE4F56A9063D1F07E714E
:10223A007F42123239201F0D7E197FFB7C717D3C53
:10224A00AB2912463390713D7404F0A3E0752C005B
:10225A00F52DA3E0FEE4EE422C7402252DF52DE4C3
:10226A00352CF52C90713E7401F0E4A3F0A3E52D12
:10227A00F0E52CA3F07F06124930852C5C852D5D94
:10228A008002C21E300C02C20620060302245BE54D
:10229A007054802438F582E43467AF82F52A8F2B94
:1022AA003021107E1A7F00E570547FFBAD2BAC2ADB
:1022BA00124633200E06200F03022459852B8285ED
:1022CA002A83A3E0FF9064D2E0FEEF6E600302244B
:1022DA0055E52B2407F582E4352AF583E0FEE52B44
:1022EA002406F582E4352AF583E07C002400F52DE6
:1022FA00EC3EF52C852B82852A83E0544F24BF605F
:10230A004D24FE60721470030223B624FB7003028C
:10231A0023CF1470030223EE1470030223EE240B5E
:10232A00600302244B201F077E1A7F06124B0FE41C
:10233A00906103F09064D2E0906104F07F02125938
:10234A00C7756155E4907137F0C22C022455201FDD
:10235A00077E1A7F1C124B0FE4906103F09064D23F
:10236A00E0906104F07F021259C7756155E49071DB
:10237A0037F0C22C022455201F077E1A7F34124BD5
:10238A000FE4906103F09064D2E0906104F07F0260
:10239A001259C7201F077E1A7F37124B0FE52B24CD
:1023AA0002FFE4352AFE123239022455201F077E25
:1023BA001A7F34124B0FE52B2402FFE4352AFE1252
:1023CA003239022455201F077E1A7F3F124B0F9085
:1023DA006103740BF09064D2E0906104F07F021202
:1023EA0059C78067201F077E1A7F57124B0F7E61DD
:1023FA007F051209028F29E5296027906103740875
:10240A00F09064D2E0906104F03005020529300BA7
:10241A000205293004020529E5292402FF1259C7B9
:10242A0080299061037409F09064D2E0906104F00D
:10243A007F021259C7201F137E1A7F61124B0F8029
:10244A000A201F077E1A7F6E124B0FC20FC20EC2DE
:01245A00067B
:01245B00225E
:103239008E2E8F2F8F828E83E0249C700302349907
:1032490024FD7003023394243A600302354B201F96
:10325900077E1A7F74124B0F852E83852F8263A2F6
:103269000190672B63A2017F0B123851852F82854C
:103279002E83A3A3E0543FF50A7403252FF52FE409
:10328900352EF52E300408052FE52F7002052E8501
:103299002F82852E83E0FF906100E0FEEF6E6003D0
:1032A90002354B052FE52F7002052E300508052F35
:1032B900E52F7002052E852F82852E83E075660025
:1032C900F567052FE52F7002052EF582852E83E01F
:1032D900FEE4EE4266052FE52F7002052E9066E8A2
:1032E900E0FEA3E0FFC3E5679FF567E5669EF56627
:1032F900D3E5679480E5669400400302354B300BB3
:1033090008052FE52F7002052E852F82852E83E073
:10331900F50CE50A64067066E50C30E742201F07E4
:103329007E1A7F79124B0F302C0302354BD22CE4D5
:1033390090711FF0906206F0E566C4F854F0C86811
:10334900E567C4540F48907120F0E567540F25E0F4
:10335900FFE433E50C640154012F907125F022201C
:103369001F077E1A7F81124B0F202C0302354B90C9
:10337900711FE06406600302354B7402F022201FBE
:10338900077E1A7F8D124B0FC22C22201F077E1A2F
:103399007F96124B0F7406252FF52FE4352EF52E47
:1033A900300508052FE52F7002052E300B08052F73
:1033B900E52F7002052E300408052FE52F70020550
:1033C9002E052FE52FAE2E7002052E14F5828E8361
:1033D900E0F50C052FE52FAE2E7002052E14F582AF
:1033E9008E83E0756700F566E50C2567F567E435BA
:1033F90066F566F562856763052FE52FAE2E7002C7
:10340900052E14F5828E83E0543FF50C052FE52F28
:10341900AE2E7002052E14F5828E83E0541FF50B33
:10342900052FE52FAE2E7002052E14F5828E83E04E
:10343900541FF50A052FE52FAE2E7002052E14F53F
:10344900828E83E0540FF50D052FE52FAE2E700205
:10345900052E14F5828E83E0547FF508AE66AF67BA
:103469007C037DE8122F318F09850C6B201F097DA4
:1034790002AF63AE62124BF71243F9907121E51165
:10348900F0A3E510F0A3E50FF0A3E50EF0D22E228C
:10349900201F077E1A7F9E124B0FE56160030235DC
:1034A9004B852F82852E83A3A3E064066003023532
:1034B9004B7406252FF52FE4352EF52E300508051A
:1034C9002FE52F7002052E300B08052FE52F70020E
:1034D900052E300408052FE52F7002052E852F8251
:1034E900852E83E06414705AE4F50C74D5250CF527
:1034F90082E43466F583E030E00E74D5250CF5825C
:10350900E43466F5837483F074C9250CF582E434D8
:1035190063F583E0FF30E40F74C9250CF582E434C8
:1035290063F583EF44A0F0050CE50CB408BD906287
:103539000874FFF090670AF0E49066E7F0C2087536
:03354900610122FB
:105A28008E318F32300404E4123861906100E01244
:105A38003861300504E4123861E532123861E53125
:0B5A4800123861300B04E412386122B8
:040902008E2E8F2F77
:10090600E56164557036201F077E1A7FA6124B0FCD
:1009160063A201852E83852F8263A201E4F56174AB
:100926004612386174011238617404123861E4FFAA
:10093600FE125A2874021238617F0722202C030205
:100946000A0F907137E0605190672B63A201852EE4
:1009560083852F8263A2017F0B123851907137E095
:10096600B40117201F077E1A7FC0124B0F852F82F6
:10097600852E83A3A3740AF08015201F077E1A7F95
:10098600C9124B0F852F82852E83A3A37447F0E4EB
:10099600907137F0C22C7F072290711FE0640570BA
:1009A60031201F077E1A7FD4124B0F90672B63A24C
:1009B60001852E83852F8263A2017F0B1238518514
:1009C6002F82852E83A3A37407F090711F14F07FE6
:1009D600072290711FE06403702F201F077E1A7F85
:1009E600E0124B0F90672B63A201852E83852F8221
:1009F60063A2017F0B123851852F82852E83A3A314
:100A06007407F090711FF0FF22E56E656D700302AA
:100A16000B0D201F077E1A7FEF124B0FE56D240882
:100A2600F5307408256DF56DD21374022530F58204
:100A3600E43460F583E0F51174032530F582E4347F
:100A460060F583E0F51074042530F582E43460F532
:100A560083E0F50F74052530F582E43460F583E014
:100A6600F50E12429E74072530F582E43460F58354
:100A7600E0FE74062530F582E43460F583E0FDEE91
:100A8600F566EDF567AF097E007C037DE8122F1F42
:100A9600EF2567F567EE3566F56663A201852E8359
:100AA600852F8263A201741E1238617401123861A7
:100AB600740312386174002530F582E43460F583DE
:100AC600E0FF9064D4E02FFF9064D3E03400FE1280
:100AD6005A2874012530F582E43460F583E0123833
:100AE60061E567123861E566123861E50C12386116
:100AF600E50B123861E50A123861E50D123861E539
:100B0600081238617F0E22E56130E045201F077E1E
:100B16001A7FF5124B0F63A201852E83852F826300
:100B2600A20174641238617401123861E561B4017E
:100B36000A74071238617561028008740A123861F6
:100B4600E4F561E4FFFE125A2874141238617F0737
:100B560022200803020C0B201F077E1B7F03124B6B
:100B66000FC20863A201852E83852F8263A20174BA
:100B76000112386174A0123861906208E024D5F53C
:100B860082E43466F583E030E1167414123861901D
:100B96006208E024D5F582E43466F583E4F0800546
:100BA6007402123861906208E075F020A4FF906428
:100BB600D4E02FFF9064D3E035F0FE125A28E4F516
:100BC60030906208E025E025E0240BF582E43467E6
:100BD600F583E5822530F582E43583F583E0F50A71
:100BE600E4F50CE50A5401123861E50AC313F50A67
:100BF600050CE50CC3940840EA0530E530C39404BF
:100C060040BF7F26229066E7E07003020DA8201FF2
:100C1600077E1B7F09124B0F9066E7E025E025E073
:100C2600F50CE4F063A201852E83852F8263A20171
:100C360090670AE0FF24C9F582E43463F583E03067
:100C4600E56374C92FF582E43463F583E4F0300973
:100C560007740B12386180057409123861E50C249B
:100C660080123861741412386190670AE075F020BA
:100C7600A4FF90620CE02FFF90620BE035F0FE12AD
:100C86005A2890670AE075F040A424D5F582E5F06D
:100C96003464F583AF0C12386AE50C75F003A4F5DD
:100CA600302406FF22200A03020FAA30121D300943
:100CB60007740C1238618005740A123861E50C2439
:100CC600801238617403123861801B300907740B77
:100CD60012386180057409123861E50C24801238D7
:100CE60061740112386190670AE075F020A4FF90E4
:100CF600620CE02FFF90620BE035F0FE125A28904E
:100D0600670AE075F040A424D5F582E5F03464F571
:100D160083AF0C12386AE50C75F003A4F530301277
:100D26007B252FF52FE4352EF52E90670AE0FF255B
:100D3600E025E024EAF582E43466F583E0F511EF78
:100D460025E025E024EBF582E43466F583E0F51032
:100D560090670AE0FF25E025E024ECF582E434669E
:100D6600F583E0F50FEF25E025E024EDF582E43488
:100D760066F583E0F50E12429EAF097E007C037D88
:100D8600E8122F1F8E668F67EF123861E5661238FC
:100D960061E50C123861E5302409FF22E5302406AE
:100DA600FF22200703020EBF201F077E1B7F1012A3
:100DB6004B0FC20763A201852E83852F8263A20192
:100DC6007425123861740112386174011238619009
:100DD60066E6E0FF90620AE02FFF906209E03400C9
:100DE600FE125A289066E6E025E025E0F530FF057C
:100DF6003074D22FF582E43463F583E0123861AFA4
:100E060030053074D22FF582E43463F583E012386E
:100E160061AF30053074D22FF582E43463F583E098
:100E2600123861AF30053074D22FF582E43463F5A1
:100E360083E0123861E412386174FC2530F530FF26
:100E4600053074C92FF582E43462F583E0F511AFFD
:100E560030053074C92FF582E43462F583E0F5106D
:100E6600AF30053074C92FF582E43462F583E0F5BE
:100E76000FAF30053074C92FF582E43462F583E094
:100E8600F50E12429EAF097E007C037DE8122F1FED
:100E96008E668F67EF123861E566123861E50C12CF
:100EA6003861E50B123861E50A123861E50D123832
:100EB60061E5081238617F1222201103020FAA2071
:100EC6001F077E1B7F16124B0FC21163A201852ED0
:100ED60083852F8263A201A2318212507B300907DB
:100EE600740C1238618005740A12386174841238E1
:100EF600617403123861906207E075F004A4FF90F4
:100F0600620CE02FFF90620BE035F0FE125A28903B
:100F16006207E075F008A424D5F582E5F03464F59F
:100F2600837F0412386A906207E025E02486F58202
:100F3600E43461F583E0F566A3E0F567123861E510
:100F460066123861906207E0240EF582E43462F599
:100F560083E01238617F1522300907740B1238615D
:100F6600800574091238617484123861740312386A
:100F760061906207E075F004A4FF90620CE02FFF19
:100F860090620BE035F0FE125A28906207E075F089
:100F960008A424D5F582E5F03464F5837F0412387D
:060FA6006A7F12227F00A9
:010FAC002222
:0100220022BB
:10511B00020FADE493A3F8E493A34003F68001F2EE
:10512B0008DFF48029E493A3F85407240CC8C33395
:10513B00C4540F4420C8834004F456800146F6DF64
:10514B00E4800B0102040810204080905BAAE47EEF
:10515B00019360BCA3FF543F30E509541FFEE49359
:10516B00A360010ECF54C025E060A840B8E493A320
:10517B00FAE493A3F8E493A3C8C582C8CAC583CA4B
:10518B00F0A3C8C582C8CAC583CADFE9DEE780BE03
:015BB00000F4
:102F1F00EF8DF0A4A8F0CF8CF0A428CE8DF0A42EC6
:022F2F00FE2280
:102F3100BC000BBE0029EF8DF084FFADF022E4CC84
:102F4100F875F008EF2FFFEE33FEEC33FCEE9DEC4D
:102F5100984005FCEE9DFE0FD5F0E9E4CEFD22ED93
:102F6100F8F5F0EE8420D21CFEADF075F008EF2FDD
:102F7100FFED33FD4007985006D5F0F222C398FDCE
:052F81000FD5F0EA226B
:102F860075F008758200EF2FFFEE33FECD33CDCC02
:102F960033CCC58233C5829BED9AEC99E582984085
:102FA6000CF582EE9BFEED9AFDEC99FC0FD5F0D662
:102FB600E4CEFBE4CDFAE4CCF9A88222B800C1B98C
:102FC6000059BA002DEC8BF084CFCECDFCE5F0CBCA
:102FD600F97818EF2FFFEE33FEED33FDEC33FCEB03
:102FE60033FB10D703994004EB99FB0FD8E5E4F9BE
:102FF600FA227818EF2FFFEE33FEED33FDEC33FCAB
:10300600C933C910D7059BE99A4007EC9BFCE99A9E
:10301600F90FD8E0E4C9FAE4CCFB2275F010EF2FE3
:10302600FFEE33FEED33FDCC33CCC833C810D707E3
:103036009BEC9AE899400AED9BFDEC9AFCE899F81E
:0E3046000FD5F0DAE4CDFBE4CCFAE4C8F922B1
:0E305400C3E49FFFE49EFEE49DFDE49CFC228D
:10306200EB9FF5F0EA9E42F0E99D42F0EC6480C8E5
:0630720064809845F02285
:10307800EB9FF5F0EA9E42F0E99D42F0E89C45F0AE
:013088002225
:10308900E493FC740193FD740293FE740393FF228D
:10309900E493F8740193F9740293FA740393FB228D
:0C30A900ECF0A3EDF0A3EEF0A3EFF0229A
:1030B500A8828583F0D083D0821230CC1230CC1216
:1030C50030CC1230CCE473E493A3C583C5F0C5833B
:1030D500C8C582C8F0A3C583C5F0C583C8C582C865
:0130E50022C8
:0C30E600A42582F582E5F03583F58322F5
:102BC300E53C2430F8E6053C22782D302A027830A3
:102BD300E475F0011231990230F22023EB7F2ED2FB
:102BE300238018EF540F2490D43440D4FF30270BA4
:102BF300EF24BFB41A0050032461FFE53D600215C2
:102C03003D0540E5407002053F302A0D782DE475FF
:102C1300F001123199EF02313802585A7403D22A63
:102C23008003E4C22AF53C8B2D8A2E892FE4F53DDF
:102C3300F53FF540E53D60077F20122BFE80F575DB
:102C43003EFFC224C223C225C226C228C229C22BE8
:102C5300122BCCFF700D302A057F00122C0FAF40D2
:102C6300AE3F22B4255FC2D5C227122BCCFF24D09E
:102C7300B40A00501A75F00A783D30D50508B6FF3E
:102C83000106C6A426F620D5047002D22680D924D4
:102C9300CFB41A00EF5004C2E5D227022E0FD2247C
:102CA30080C6D22380C0D22580BCD2D580BAD22898
:102CB30080B47F20122BFE2025077401B53D004010
:102CC300F1122BC3FF122BFE022C37D22BD22980F9
:102CD30095122BC3FB122BC3FA122BC3F94A4B7069
:102CE3000679E07A2E7BFF20252EE53D602A7E00C3
:102CF3008E8275830012310B60060EEE653E70F016
:102D0300C2D5EBC0E0EAC0E0E9C0E0EE122E56D037
:102D1300E0F9D0E0FAD0E0FB1230F2FF60AAEBC09A
:102D2300E0EAC0E0E9C0E0122BFED0E02401F9D0D4
:102D3300E03400FAD0E0FBE53E0460DCD53ED98008
:102D4300877BFF7A2E7952D225809C791080027975
:102D530008C229C22B8008D2D5790A8004790AC215
:102D6300D5E53E047002F53EE4FAFDFEFF122BC3E7
:102D7300FC7B08202413122BC3FD7B1030230A1283
:102D83002BC3FE122BC3FF7B20EC3382D592D5508D
:102D930013C3E43023069FFFE49EFEE42024039D37
:102DA300FDE49CFCE4CBF8C224EC700CCFCECDCC7C
:102DB300E824F8F870F38017C3EF33FFEE33FEED2A
:102DC30033FDEC33FCEB33FB994002FB0FD8E9EB0B
:102DD300302405F8D0E0C448B224C0E00AEC4D4EDC
:102DE3004F78207B0070C2EAB53E0040BCC0E012C1
:102DF3002E58D0F0D0E0202404C4C0E0C4B224C0D4
:102E0300F0122BE7D0F0D5F0EB022C371231F82C6F
:102E1300D4532D4E582CA54C2CA1422D524F2D5A34
:0F2E2300442D5A492CBA432D60552D44462D4459
:102E3200452D44472F00502CA92D2CAD2E2CD02BE4
:102E42002CB1232CCE202EE92A2C694800002CC854
:102E52003F3F3F00790AA2D5202614302809B91035
:102E6200020404B9080104A2D52029025001042059
:102E720025689225B53D005034C0E07F20302619E8
:102E82007F30A22572297228500F122EAFC225C29E
:102E920029C228C22B7F30800F302803E9C0E012FC
:102EA2002BFE302803D0E0F9D0E0B53DCC30281716
:102EB2007F30B9100C122BFE7F583027077F7880A5
:102EC20003B90803122BFE3025057F2D022BFE7F4E
:102ED20020202BF87F2B2029F322922580CF286EE9
:102EE200756C6C2900D224122BC33024F8C22478CA
:102EF2003D30D50108F6022C692D50434958122B5A
:102F0200C32403B405004001E4902EFB93122BEF7F
:0D2F1200743A122BEFD226753D04022D4EAD
:103B33008B288A29892AE4F534F533F532F531F5F2
:103B43002FF530E52C452D452B6012EBC0E0EAC084
:103B5300E0E9C0E0AB2BAA2CA92D1231A9AB2805B3
:103B63002AE52AAA297002052914F91230F2F5353B
:103B7300C394094007E535D3940D40E1E53564204E
:103B830060DBE535B42D054330038016E535B42BF2
:103B930005433001800C74FF252AF52A74FF35296B
:103BA300F529E52E60046410703FAB28AA29A92AE1
:103BB3001230F264306009E52E702E752E0A8029CA
:103BC30090000112310BFF64786004EFB458134383
:103BD3003001752E107402252AF52AE43529F529BA
:103BE3008007E52E7003752E08AB28052AE52AAA5F
:103BF300297002052914F91230F2F535C394614096
:103C03000AE535D3947A50035335DF74D02535F55F
:103C130035C3940A400CE5359411406D74F925358C
:103C2300F535E535D3952E5060433001853439851C
:103C33003338853237853136AF2E7E00E4FCFDAB59
:103C430034AA33A932A83112314AC8ECC8C9EDC924
:103C5300CAEECACBEFCBE4FCFDFEEB2535F534EE23
:103C63003AF533ED39F532EC38F531AF34AE33ADE7
:103C730032FCAB39AA38A937A836D31230785003AF
:103C8300023BEC433004023BECE53020E003E480EC
:103C93002DE52C452D452B601EAB28E52A24FFF985
:103CA300E52934FFFAEBC0E0EAC0E0E9C0E0AB2B62
:103CB300AA2CA92D1231A9E53030E20774FFFFFECB
:103CC300FDFC22E530AF34AE33AD32AC3130E1032D
:043CD3000230542245
:1030F200BB010689828A83E0225002E722BBFE02DC
:09310200E32289828A83E493220E
:10310B00BB010CE58229F582E5833AF583E0225079
:10311B0006E92582F8E622BBFE06E92582F8E222C3
:0D312B00E58229F582E5833AF583E49322DD
:10313800BB010689828A83F0225002F722BBFE0176
:02314800F32270
:10314A00E88FF0A4CC8BF0A42CFCE98EF0A42CFC24
:10315A008AF0EDA42CFCEA8EF0A4CDA8F08BF0A4A2
:10316A002DCC3825F0FDE98FF0A42CCD35F0FCEB01
:10317A008EF0A4FEA9F0EB8FF0A4CFC5F02ECD39C6
:0F318A00FEE43CFCEAA42DCE35F0FDE43CFC2233
:10319900FAE6FB0808E6F925F0F618E6CA3AF62237
:1031A900BB011A89828A83D0F0D0E0F8D0E0F9D047
:1031B900E0FAD0E0FBE8C0E0C0F00232275016E99F
:1031C900F8D083D082D0E0F9D0E0FAD0E0FBC08219
:1031D900C08302321EBBFE16E9F8D083D082D0E04C
:0F31E900F9D0E0FAD0E0FBC082C083023230227E
:1031F800D083D082F8E4937012740193700DA3A366
:1032080093F8740193F5828883E473740293686079
:06321800EFA3A3A380DF79
:09321E00EBF608EAF608E9F622D5
:09322700EBF0A3EAF0A3E9F022A8
:09323000EBF208EAF208E9F222CF
:00000001FF
